:10000000A0011D299000240884002208A520841343
:100010000005181C2206031920281008031D1828A3
:100020001608FF3E031C21280A30BE20160821288E
:10003000100AFF3003192028100B20281708212848
:100040009909031019180314182991019000A11798
:1000500027308F001030382003308F00E8303820F0
:100060008F01643038208F010A303820100843286F
:100070008E0011088D0010088C00E0200C08031D74
:10008000A113A11B0800303EA0186F289300861111
:100090008316861183123A308D009830CC2086105A
:1000A0008316861083123330920083160F30860534
:1000B000831283200F308D00DC30CC2083203C3035
:1000C000CB20832022309200832020306E200C3001
:1000D0006E2006306E20A01413086F2820149200A2
:1000E000201C7D288610033C031C822882203E3081
:1000F0008D008030CC20031408002014FE3C03192E
:1001000018298614201C20100F3086051208F0399B
:1001100086048615920E8611201883282830CB205D
:1001200003140800A200A8200C080D0403191829C4
:10013000122184132208800664009E289F288C0ABE
:1001400003198D0F9C28800618298417800418290C
:10015000FF3A841780051829890083160814831232
:100160000808182988008316081555308900AA3018
:10017000890088148818BA28081118298F018E0060
:10018000FF308E07031C8F07031C182903308D00D6
:10019000DF30CC20C0288D01E83E8C008D09FC307A
:1001A000031CD5288C070318D2288C0764008D0FF8
:1001B000D2280C18DB288C1CDF280000DF28080060
:1001C00010309200910190010D0D900D910D0E08CF
:1001D00090020F08031C0F0F91020318F6280E0857
:1001E00090070F0803180F0F910703108C0D8D0D4A
:1001F000920BE4280C081829103094008D018C0112
:10020000930C920C031C0A290E088C070F08031884
:100210000F0F8D078D0C8C0C910C900C940B0029FA
:10022000100818298C098D098C0A03198D0A0800F9
:1002300083130313831264000800831605148514C6
:10024000051683122030B4000330B50086108316E3
:100250008610831206108316061083120611831669
:1002600006118312851183168511831206118316D8
:1002700006118312C4015230B800B9016430BE20A7
:10028000FE3044200130442052304420533044207A
:10029000393044203030442034304420323044203F
:1002A0002030442020304420763044202030442028
:1002B000333044202E304420343044202030442039
:1002C00031304420303044204D30442003308F0002
:1002D000E830BF20DA290530A4001030A2009801D0
:1002E000FF30960097010130990041080220C100BB
:1002F0000318BC290530A4000130A20098010A307F
:10030000960002309700013099003D080220BD00A0
:100310000318052A0530A4000230A20098010A3013
:10032000960002309700013099003E080220BE007E
:100330000318132A0530A4000430A2009801FF30EE
:1003400096009701013099003F080220BF00031872
:10035000852A0530A4000430A20001309800FF3047
:10036000960097010130990040080220C000031850
:10037000412A6430BE206B290430C4076400093070
:1003800044020318C429C529C40164004408043C7C
:100390000319D32964004408083C0319D7295230B3
:1003A000B800B901DA294430B800B901DA2953306C
:1003B000B800B901003044079E009F019F0D1E0840
:1003C000AC20BC00013044079E009F019F0D1E0819
:1003D000AC20B200B301C830B2070318B30A023030
:1003E00044079E009F019F0D1E08AC20BB000330F8
:1003F00044079E009F019F0D1E08AC20B000B10174
:10040000C830B0070318B10A412A64003C087F3C99
:100410000319212ABC0A64003B087F3C0319272AE0
:10042000BB0A0123412A64003C08003C03192D2A21
:10043000BC0364003B08003C0319372ABB030123BB
:10044000412AB20A0319B30ABC0114230B2AB00AC9
:100450000319B10ABB011423112A0130B202003082
:10046000031C013EB3027F30BC001423192A013063
:10047000B0020030031C013EB1027F30BB001423E8
:100480001F2A5230B600B7013C08BA0001303207CB
:10049000AC0033080318013EAD00061083160610A9
:1004A00083123F2332308C008D01063084000130EE
:1004B00092203B08BA003008AC003108AD0085112D
:1004C0008316851183123F2332308C008D01053055
:1004D000840008309220CF303002AE000030031C80
:1004E000013E3102AF0064303B079E009F019F0D2B
:1004F0007D30920093011E088E001F088F00FC20A3
:10050000A8001108A900C5226B295430B600B70114
:100510003B08BA0001303007AC0031080318013E37
:10052000AD0085118316851183123F2332308C0074
:100530008D0105308400083092203C08BA00320852
:10054000AC003308AD0006108316061083123F235B
:1005500032308C008D010630840001309220FA3058
:100560003202AE000030031C013E3302AF007D308A
:10057000920093013C088E008F01FC20A800110816
:10058000A900C5226B296300C32A403092000630BF
:1005900093002E088E002F088F00FC20A600110863
:1005A000A70028088C0029088D000A308E008F01D2
:1005B000E0209E000D089F0026081E07AA002708BD
:1005C0000318013E1F07AB00FE30442001304420D9
:1005D0003608442058304420203044200430252060
:1005E0002B0891002A082620203044206B3044201C
:1005F000483044207A3044202030442038084420B9
:100600000800003044079E009F019F0D1E088900CE
:100610003C08B220023044079E009F019F0D1E0837
:1006200089003B08B2200800003044079E009F016B
:100630009F0D1E0889003C08B220C8303202C3005A
:10064000013044079E009F019F0D1E08890043084A
:10065000B220023044079E009F019F0D1E088900B2
:100660003B08B220C8303002C200033044079E006D
:100670009F019F0D1E0889004208B2200800B51A8C
:100680000615B51E0611E423351A0615351E06118A
:10069000E423B5190615B51D0611E4233519061511
:1006A000351D0611E423B5180615B51C0611E42303
:1006B00035180615351C0611E423B41B0615B41FA6
:1006C0000611E423341B0615341F0611E423B41A63
:1006D0000615B41E0611E423341A0615341E06113D
:1006E000E423B4190615B41D0611E42334190615C4
:1006F000341D0611E423B4180615B41C0611E423B6
:1007000034180615341C0611E423AD180615AD1C6B
:100710000611E4232D1806152D1C0611E423AC1B2D
:100720000615AC1F0611E4232C1B06152C1F061101
:10073000E423AC1A0615AC1E0611E4232C1A061588
:100740002C1E0611E423AC190615AC1D0611E4237A
:100750002C1906152C1D0611E423AC180615AC1C2B
:100760000611E4232C1806152C1C0611E4233A1B51
:1007700006153A1F0611E423BA1A0615BA1E061109
:10078000E4233A1A06153A1E0611E423BA1906158F
:10079000BA1D0611E4233A1906153A1D0611E42381
:1007A000BA180615BA1C0611E4233A1806153A1CA5
:1007B0000611E4230615831606118312E42306119D
:1007C000831606118312080005308C008D01063057
:0807D0008400023092200800B1
:02400E00F53F7C
:10420000620044007E001900620045007E00180034
:084210000800470024001B0018
:00000001FF
